:10000000709D0010ED010000F5010000F7010000F7
:10001000F9010000FB010000FD010000C656FFEFE2
:10002000000000000000000000000000FF010000D0
:100030000102000000000000030200006502000051
:100040000702000011020000070200000702000082
:10005000070200000702000007020000070200007C
:10006000070200000702000007020000070200006C
:100070000702000000000000070200000702000065
:10008000070200000702000007020000070200004C
:10009000070200000702000007020000070200003C
:1000A0008924000007020000070200000702000088
:1000B000070200000702000007020000070200001C
:1000C000070200000702000007020000070200000C
:1000D00007020000070200000702000007020000FC
:1000E00007020000DFF80CD004F0FCFD00480047D8
:1000F0008B090000709D0010D0F800D0D0F804F0FB
:1001000070B50023084D0AE0CE5C048886EA142608
:1001100035F8166086EA042404805B1C9BB2521EEC
:1001200092B2F1D270BD0000484F0000FFB5044606
:1001300029A090E8E000C0688DE8E0000390022963
:1001400002DA002004B0F0BD6018002100F8011DA3
:100150006946B3FBF2F502FB15354D5D00F8015D14
:10016000B3FBF2F3A042F4D8ECE710B504F0F7FCCF
:1001700004F0E0FC1C4948604FF480520A60A0F58E
:10018000F420886010BD70B5034608460024164967
:10019000851849688D4200D9881A194604F02FFD48
:1001A000204670BDF8B50346104600240A460E4DA1
:1001B000161869688E4200D90A1A0090286804F05F
:1001C0004AFD2046F8BD10B50346084600241946EE
:1001D00004F0E8FC204610BD303132333435363778
:1001E0003839414243444546B40000100648804730
:1001F00006480047FEE7FEE7FEE7FEE7FEE7FEE70C
:10020000FEE7FEE7FEE7FEE791180000E5000000CC
:1002100010B54FF040210120086000F0CEF810BD6D
:1002200010B54FF0E0241A4860611F21601700F0FC
:100230001EF80020A0610720206110BD10B51548F0
:10024000022141600021016741611D22C260C1633A
:1002500001214160FFF7E4FF0221C81E00F007F80A
:10026000002010BD0C480168491C01607047C90698
:10027000090E002806DA00F00F0000F1E02080F8F7
:10028000141D704700F1E02080F800147047000052
:10029000BFD4010000000940E800001010B50B4673
:1002A00004461146184600F015F8C4E9000110BDD7
:1002B00040EA01039B0703D009E008C9121F08C0E8
:1002C000042AFAD203E011F8013B00F8013B521E68
:1002D000F9D2704770B500242546002801DA0124C0
:1002E0004042002901DA0125494204F00DFDAC42EB
:1002F00000D04042002C00D0494270BDFFFFFFFFFC
:10030000394800210167C1600222426181613022C7
:10031000C2633648826836480260416000207047F8
:1003200070B541F28832904208D8642800D228B9CA
:1003300042F21072914201D8052901D2002070BD0D
:100340002A4DAA682A4B1C68141B5A6802EB420605
:10035000C6EBC212B4EBC20F01D2002070BD224A1C
:100360000224546038B1234EB6FBF0F04010906187
:10037000546001205060A86818605960002070BD6A
:1003800070B50C461A4D00266E602146FFF7C8FF77
:1003900004EB4400C0EBC411144A286893681B1A8C
:1003A000B3EBC10FFAD3104802214160C16B01F0D9
:1003B000FE01C1636E60002070BD0C4880680C496E
:1003C0000A68821A486800EB4003C3EBC010B2EB26
:1003D000C00F08D3044802224260C26B02F0FE0242
:1003E000C263002048607047008000400000094060
:1003F000EC00001080C3C90170470000000000003D
:10040000000000008609000010B5FB4C6069800404
:100410000CD4FA48816843F6982283685B1A9342A9
:10042000FBD36069800401D4012010BD052001F0D8
:1004300037F8002010BD2DE9F0410024EF4EB568DB
:10044000042001F02DF8EE4F02E0FFF7DDFF30B1A0
:10045000B068401BB842F8D3012C02D00CE0012454
:10046000FAE7022404E0FFF7CFFF08B1032403E01A
:10047000B068401BB842F6D3032C02D00020BDE880
:10048000F0810120FBE72DE9F041092001F008F897
:10049000DC48002606704FF47A77C8213846FFF70B
:1004A0006FFFD64CA16842F21075A068421AAA42AA
:1004B000FBD3C8213846FFF763FFA168A268501A32
:1004C000A842FBD3C8213846FFF75AFFCD48401C4D
:1004D000867002214171C670D1E70021425C12B9D9
:1004E000491C1829FAD3182901D00020704701208F
:1004F00070472DE9FC4107460E46904600200190CA
:1005000000240EE0351B402D00D9402539192A461C
:10051000BD48FFF758FEAAB2BB4901A8FFF7F0FD9E
:100520002C44B442EED3391942466846FFF74BFEDD
:10053000BDF80400BDF80010884202D10120BDE8DA
:10054000FC810020FBE71FB5002746208DF8000046
:100550004FF000098DF8039036208DF8010033200C
:100560008DF80200A94908684FF6FF021040A84A1A
:1005700040F4807010430860A648C0F80090A64878
:100580006FF4305100680844A4490860A44900F59C
:10059000E0500860A349400A0860A34CF82020708E
:1005A000FF206070A070FFF7ABFE0020954E9F4AC1
:1005B000761C96F9041052F82110221802F5805288
:1005C0000B5C82F80038401C6028F6D34FF4E174CD
:1005D000214640F24910FFF7D3FE214640F29F101A
:1005E000FFF7CEFE4FF48054DFF844A24FF001082D
:1005F000307808B101F0D2FF707928B101287CD0A1
:10060000307800287AD0AFE10A2000F049FF1922A3
:1006100021468748FFF7D7FD022216212046FFF723
:1006200068FF00286BD0DAF80E10022204F11900DE
:10063000FFF75FFF00287DD09AF80020062A29D214
:10064000DFE802F02A2A032A2A177A4BDAF80A008E
:10065000596F491C884209D25B6F1D1ADAF80E30B7
:100660006D1C9D4202D31844884215D986F8028039
:1006700012E0DAF80E00B0F5F42F01D986F8028006
:10068000DAF81200C0F30B40B0F5107F04D086F802
:10069000028001E086F80280022A01D0052A46D1B4
:1006A000CDF80C90022204F21D4103A8FFF78BFD48
:1006B0000399DAF8040089B2884201D086F80280F2
:1006C000CDF80C90012204F2254103A8FFF77BFD31
:1006D0000399BAF80100C9B2884201D086F80280B5
:1006E0009AF80000022822D1CDF80C90042204F2DE
:1006F000494103A8FFF767FD02E05BE02DE148E018
:10070000DAF812000399884201D086F80280CDF809
:100710000C90012204F24D4103A8FFF754FD039908
:100720009AF80300C9B2884201D086F802809AF88C
:10073000180000E02AE0401EFE2801D286F8028060
:10074000BAF80100A0F57F41FF3901D03F2802D15E
:100750009AF8030028B93648FFF7BFFE08B986F8B3
:100760000280DAF80E001B3404443148FFF7B5FE6E
:1007700088B14FF4805486F8058086F803900620EF
:1007800000F08EFE0A2000F08BFE04E086F8028066
:1007900001E086F80280F078401CC0B2F0700C28AE
:1007A00001D386F80280B07800283FF421AFFFF72C
:1007B0006AFE1DE7192221461D48FFF704FD9AF83D
:1007C0001800C0B19AF80000062814D2DFE800F043
:1007D00082030555575901277CE001279AF8090043
:1007E000012877D1DAF80A0018B913488069CAF8E5
:1007F0000A0000253CE06DE000800920000009406F
:1008000080841E00680000104D1B00100CED00E0FD
:100810000000FA05B0000010BC000010A00000109D
:10082000980000109C0000104D01001060000010A6
:10083000340100100053000088520000072000F02F
:100840002FFEDAF80E00A0EB050BBBF1400F01D92B
:100850004FF0400B611919315A467E48FFF7B3FC3F
:10086000DAF80A005A4628447A4900F082FD5D44CD
:10087000DAF80E00A842E1D82CE001272AE001278F
:1008800028E001279AF80900032823D17248734908
:1008900000680860002519E0072000F001FEDAF882
:1008A0000E00A0EB050BBBF1400F01D94FF0400B40
:1008B000611919315A466748FFF785FC66485A4660
:1008C000006841196348FFF76DFC5D44DAF80E00DB
:1008D000A842E1D89AF8180070B19AF8000058B10F
:1008E0008AF81890192221465D48FFF74CFCC82170
:1008F0004FF47A70FFF744FDDAF80E001B3404441D
:100900005748FFF7EAFDC8B14FF4805402207071D8
:10091000544880F800900B2000F0C2FD77B100270A
:100920005148816842F2107283685B1A9342FBD38C
:100930004FF42F714FF47A70FFF722FDF078401CCE
:10094000C0B2F0700C2801D386F80280B07800287D
:100950003FF42FAFFFF797FD4AE686F8008001F0DD
:10096000ACFC012001F06AFC3E4800780028F3D07E
:100970000021684600F022FC0028EDD04FF480549E
:1009800086F8059086F8039032E636484FF0000866
:10099000C0F80180A0F80580324FFF207F1C38711D
:1009A00087F8058000F074FF00F0C2FFFFF746FCF7
:1009B00000F03AFD002000F073FD01F055FE2B4ED3
:1009C0007069400302D5FFF71FFD48B300240420DF
:1009D00000F066FD7069244D800416D4FFF72BFDEE
:1009E000A0B1FFF728FD88B1FFF725FD70B1042005
:1009F00000F056FD0124A8681D497269920405D4CF
:100A0000AA68121A8A42F8D300E0012444B1A86807
:100A100042F21071AA68121A8A42FBD387F8048046
:100A200000F0DDFC58B1022000F03AFD97F9040017
:100A3000401C01D100F0CDFC0120787006E00220BE
:100A400000F02EFD87F8018087F80480FFF78DFB0A
:100A5000FFF779FD4D1B0010BC000010B400001022
:100A600034010010680000100000094000800920D7
:100A700080841E0030B50023FE4A146A2CE0B0F5D5
:100A8000007F1AD213280CD014280CD0B0F5FF7FA9
:100A90000CD0A0F58072FF3A0AD03E280AD9002275
:100AA00016E0E2B214E0C4F3072211E055220FE091
:100AB000AA220DE0F04A125C0AE0B0F5E05F06D22F
:100AC000EE4A0244A2F5805292F8002E00E0002285
:100AD000EB4DEA54401C5B1C8B42D0D330BD70B54B
:100AE000E44D2C6B402C00D94024E86AE9690219D6
:100AF0008A4202D90C1A042169702146FFF7BAFF15
:100B00002246DF49822001F098FCE86A2044E8622E
:100B1000286B001B2863DA499F318A68121B8A60A0
:100B200008B9032068706878022801D00020087393
:100B300070BD10B5D249D3489F3108600D22822084
:100B400001F07BFCCB490520487010BD70B50E4606
:100B5000CD494A69520302D5496D490521D4B0F502
:100B6000007F1ED3C949C34CB0F5E05F1AD28B6831
:100B7000A2699A1AC64B9A4204D38968A1610021DE
:100B8000616061610023BE4CBC4D403407E0C11878
:100B90002944A1F58051E25C81F8002E5B1CB34230
:100BA000F5D370BD626922B98A68A2618A68626100
:100BB000A060B84A1279002AF3D18A686369D21A10
:100BC000B54B9A421CD2B54B01221A708A68A261B9
:100BD00089686161A168401A6168884203D9616AC5
:100BE000884200D26060062000F05AFC61683246FC
:100BF000BDE87040A24801F580514030FFF7D2BAFD
:100C0000BDE870400C2000F04BBC10B5994CA178A9
:100C1000E06A4218E1698A4206D9081AA0700520E4
:100C20006070022001F0C4FBA178E06AFFF78EFF3C
:100C3000A078E16A0144E162216B091A2163904ABC
:100C40009F329368181A906011B16078052804D11A
:100C500000201073BDE810406BE710BD2DE9F04196
:100C6000844CA178E06A4218E1698A4206D9081AE0
:100C7000A07005206070022001F09AFB0020804DDA
:100C8000A17805F14003E26A08E016181F5CAE5D2A
:100C9000BE4202D00020A06202E0401C8842F4D391
:100CA0005018E062206B401A2063754A9F329368A7
:100CB000591A916010B16078052808D1A06A20B156
:100CC00000201073BDE8F04133E70120F9E7BDE8EB
:100CD000F08110B56A488030017D427CC37C41EAD6
:100CE0000261827C120442EA03221143614A4902F2
:100CF000D162C17D837D41EA03214902116380688D
:100D000088420DD0822001F053FB022001F050FBFD
:100D10005B4902209F310873FFF70BFF002010BDD5
:100D2000012010BD70B556480225803000F11F0427
:100D3000816800290AD0007B00060CD4022001F053
:100D400037FB2573FFF7F5FE002070BD2573FFF715
:100D5000F0FE002070BD012070BD10B54848454C24
:100D600080308068A178884200D2A0704449A2787F
:100D70004031822001F061FB032060704048A2787E
:100D80009F308168891A81600021017310BD10B500
:100D90003B4880308168002909D0007B000603D5DC
:100DA000822001F005FB02E0022001F001FB344942
:100DB00000209F310873BDE81040BAE610B5FFF778
:100DC000B1FF00281FD02E48702140300170002153
:100DD000417002228270C1700171417181710A22D9
:100DE000C271017241728172C1723022027301229A
:100DF00042738173C173017441741E49122088705B
:100E0000BDE81040A9E710BD1CB5FFF78BFF002817
:100E100068D023480A22062103886846FFF786F92E
:100E200017480022403002708023437082700121F5
:100E3000C1702021017143718271C271412202721D
:100E4000542242724F2282724C22C2720173417349
:100E50008173C173462202745023437472238374D6
:100E60006923C3746E230375742343758175C2753A
:100E70006C2217E07C000010485200004D01001069
:100E80004D1B0010555342530080092000000940BB
:100E9000A08601006900001020A107006800001072
:100EA0000404000002766122427673228276682270
:100EB000C276017741778177C1779DF8011080F87C
:100EC00020109DF8021080F821109DF8031080F882
:100ED00022109DF8041080F82310E849242088701F
:100EE000FFF73BFF1CBD10B5FFF71CFF00280CD01F
:100EF000E34803210170002141708170C170DF4916
:100F000004208870BDE8104027E710BD10B5FFF73A
:100F100009FF002810D0DA48002101700622427033
:100F20008170C170017141718171C171D349082013
:100F30008870BDE8104010E710BD10B5FFF7F2FE55
:100F4000002815D0CD4ACE48116A491E0B0E0370F9
:100F50000B0C43700B0A8370C17000210171417149
:100F600002238371C17108209070BDE81040F4E63F
:100F700010BD10B5FFF7D6FE002819D0C0480022DA
:100F80000270427082700821C170BC4B196A0C0E4D
:100F900004710C0C44710C0A8471C171022101723C
:100FA00042728172C2720C209870BDE81040D4E683
:100FB00010BD2DE9F0410020B04DB14CB04AA978E8
:100FC000403402E0135C2354401C8842FAD31F29AA
:100FD00078D12168AB4881427CD1A94E60685F36E8
:100FE0007060A068B060607B4FF0010818B9A07B0A
:100FF00008B1102804D986F80C80BDE8F04198E5C6
:10100000E07B1E28F7D00FDC12282ED005DC48B379
:101010000328F0D1BDE8F041D0E61528EBD01A281E
:10102000E9D1BDE8F0415EE702272A282DD010DC87
:1010300023281DD025281ED02828DCD1FFF749FE03
:1010400000282BD0207B000618D56F70BDE8F0413A
:1010500045E52F282AD05528CDD05A28CBD1BDE838
:10106000F04153E7BDE8F04191E6BDE8F041CBE641
:10107000BDE8F0417DE7BDE8F0415EE7022001F008
:1010800097F93773BDE8F04153E5FFF722FE0028DA
:1010900004D0207B000602D485F8018017E6822068
:1010A00001F086F93773BDE8F04142E5FFF711FE24
:1010B0000028F3D0207B000605D485F80180C5F810
:1010C000288004E606E0822001F072F93773BDE85B
:1010D000F0412EE5822001F06BF9022001F068F961
:1010E00006206870F3E510B564494878022808D0F6
:1010F00003280ED004280FD0052801D10020487005
:1011000010BD5F484030C07B2828F9D1BDE81040B1
:10111000E5E4BDE810400CE5822001F049F9BDE8A6
:10112000104006E510B55649022001F055F9534923
:101130008870487858B101280CD0022001F038F9A5
:101140004F4902205F310873BDE81040F1E4BDE86B
:1011500010402EE74A484030C07B2A2804D02F2870
:1011600005D1BDE8104079E5BDE810404DE510BD62
:10117000FFB502460020002102EB42064FF4405723
:1011800001AD6C46721845F82120BA4202DD0020FC
:1011900004B0F0BD3C4B03EB62031B786354D207F1
:1011A00001D01A096254625C02F00F0262548B0093
:1011B0009A401044491C0329E4DBE9E7F0B50646F0
:1011C000002000220023304F4FF4007C52E0521CDC
:1011D000B45C3CB19D183D4405F5805595F8005828
:1011E000A542F4D0032A44D303F5C0503A18107F27
:1011F000547FD57F00EB0420947F240404EB056426
:10120000204451EA000401D011B108E00020F0BDF3
:101210001A4949684031884201D90020F0BD0020B8
:1012200017496C311C183C4404F5805494F800486C
:101230000C54401C0C28F5D3907ED17E00EB01208D
:10124000117D527D090401EB026145182846FFF724
:101250008FFF40F6F57401E0FFF78AFFC11EA1423F
:10126000FAD3A0F57061FF3901D00020F0BD284607
:10127000F0BD20336345ABD3F0BD00007C0000100F
:101280008D1B0010555342434D01001062B670474C
:1012900030B45E4A5D4C032328342360136843F462
:1012A000803313605A4A30BC104772B6704770B52D
:1012B000054600242046FFF7F8FF564B3320186000
:1012C0005D609960DA6054484FF47A710068B0FB51
:1012D000F1F0186103F114011846FFF7D9FF204619
:1012E000BDE87040D2E74B4A3223136050609160F2
:1012F00049484FF47A710068B0FBF1F0D06002F118
:1013000014011046C4E7434A3423136050609160CF
:1013100041484FF47A710068B0FBF1F0D06002F1FF
:1013200014011046B4E770B5014600252846FFF7C2
:10133000BCFF0624394850F824208A4212D9374885
:10134000783850F82400884207D121462046FFF71C
:10135000CAFF21462046FFF7D6FF21462046FFF769
:10136000C2FF02E0641C1D2CE5D92846BDE8704090
:101370008CE72DE9F0412A4C2368002B00D1206036
:101380000020274B234D5B68283503E01F180E5CB7
:10139000EE55401C9042F9D3981860604FF4807667
:1013A000B04213D12068FFF7BEFF1A4D14352868EC
:1013B00000B1FEE71749324628312068FFF777FF72
:1013C000286800B1FEE70020606020600020BDE8D2
:1013D000F08114494FF4C0400860FEF78DBE002133
:1013E00046F204400088A0F51942993A0AD04FF419
:1013F000C0404FF4002304C811449842FBD319B1F4
:1014000000207047012070470120704788C10F40BD
:10141000F11FFF1F081C0010D8000010005300002F
:10142000C000001008ED00E0002070479749C20797
:1014300002D04FF000728A67800702D54FF08060BB
:101440008867002070479149C20702D04FF00072B0
:10145000CA67800702D54FF08060C86700207047D8
:1014600000218A4AC30703D0536F9B0100D5012195
:10147000800704D5506F400101D541F0020188B2C8
:10148000704710B504462046FFF7EAFF03461846AA
:10149000FFF7D9FF24EA0300FFF7C8FF002010BDC3
:1014A000F0B503467A4C002B0AD060680425032669
:1014B0000227052807D2DFE800F0073869A6D10027
:1014C00000206060A060F0BD042B02D0052B07D087
:1014D00009E00320FFF7B7FF0120FFF7A7FF02E0B5
:1014E0000120FFF7B0FF0125022B0ED0012B14D0F5
:1014F0000E2BE8D10320FFF7A6FF0220FFF796FF8F
:101500000120FFF793FF6560F0BD0320FFF79BFF0D
:101510000220FFF78BFF6560F0BD0320FFF793FF0C
:101520000120FFF783FF6560F0BD062B10D0032B71
:1015300016D00A2B1CD0092B1AD00D2B1FD00C2B28
:10154000F2D10320FFF77FFFBDE8F04001206DE7F7
:101550000320FFF778FF0220FFF768FF6760F0BD08
:101560000320FFF770FF0120FFF760FF6660F0BD0A
:101570000320FFF768FFBDE8F040022056E7032094
:10158000FFF761FFBDE8F04002204FE7062B13D0C4
:101590000A2B1AD0092B20D00C2B26D00D2B2BD0A8
:1015A0000F2BE4D10320FFF74EFF0220FFF73EFF91
:1015B000BDE8F040012039E7A068411CA160C006E9
:1015C000D5D1BDE8F04002205BE70320FFF73BFFE9
:1015D0000220FFF72BFF6660F0BD0320FFF733FF0B
:1015E0000120FFF723FF6560F0BD0320FFF72BFF0D
:1015F000BDE8F040012019E70320FFF724FFBDE814
:10160000F040022012E7072B0DD00A2B17D00B2B2E
:101610001CD0092BE8D10320FFF715FF0120FFF7AD
:1016200005FF6560F0BD0220FFF70DFFA068411CBB
:10163000A1608006F6D1BDE8F040012021E703203B
:10164000FFF701FFBDE8F0400120EFE60320FFF7C0
:10165000FAFE0220FFF7EAFE6560F0BD062B0CD013
:101660000E2BFAD10320FFF7EEFE0220FFF7DEFE7D
:101670000120FFF7DBFE6560F0BD0320FFF7E3FE0E
:101680000220FFF7D3FE6760F0BD00000080092054
:10169000CC000010F0B5A14DD5F804014FF00002C8
:1016A000C1059F4852D4D5F80C119E4BC90707D0ED
:1016B000D5F8A011490626D40260426082609EE0FF
:1016C000D5F80411C9061AD0D5F8041101F01F018C
:1016D000B3FBF1F10160D5F8A841E40611D0D5F8CB
:1016E000A84104F01F04B3FBF4F34360D5F80031C4
:1016F00003F001035B1CB1FBF3F181607FE000218B
:10170000E8E70023F1E7D5F80411C9061AD0D5F8A7
:10171000041101F01F01B3FBF1F10160D5F8A841FC
:10172000E40611D0D5F8A84104F01F04B3FBF4F38C
:101730004360D5F8003103F001035B1CB1FBF3F10A
:1017400081605CE00021E8E70023F1E7D5F888102C
:10175000C90503D402604260826050E0D5F80C11E4
:10176000C90707D0D5F8A011490628D40260426005
:10177000826044E055F8881F01F01F035B1CE96F8D
:1017800001F01F01D5F8204104F01F04AE6F883D21
:1017900006F00106761C71B1624F5F43B7FBF1F1B1
:1017A000016054B15F4F7B43B3FBF4F34360B1FB83
:1017B000F6F1816023E00021F2E70023F6E755F817
:1017C000881F01F01F035B1CE96F01F01F01D5F8B2
:1017D000204104F01F04AE6F883D06F00106761C20
:1017E000E1B1504F5F43B7FBF1F10160C4B14D4F20
:1017F0007B43B3FBF4F34360B1FBF6F18160D5F8B2
:101800000811C90528D5D5F8081111F01F0109D014
:10181000042909D0062907D0C260F0BD0021E4E701
:101820000023E8E7C260F0BD903555F8081C01F0D0
:101830001F01491CAA6F02F01F02EB6FDB0705D0E6
:10184000384B5943B1FBF2F1C160F0BD354B594300
:10185000B1FBF2F1C160F0BDD5F80811890515D5CD
:10186000D5F80C11C90708D0D5F8A8102D4A01F0F9
:101870001F01491C5143C160F0BDD5F88810294AA9
:1018800001F01F01491C5143C160F0BDC260F0BDB1
:1018900010B422482021C0F8A011D0F8A0114906A8
:1018A000FBD501228030C0F88C2009214160026004
:1018B000AA24C4605523C3608038D0F88810490535
:1018C000FBD52321A03041600260C460C360A03812
:1018D000D0F8A8104905FBD58C3040F20111816782
:1018E00040F20121C16742670221C0F8281104219A
:1018F000C0F81C110C4981630021C0F83C11D0F8DC
:10190000242142F00302C0F8242145F23A0240F8B3
:101910008C2C0648016010BCBCE6000000C00F40E3
:10192000D8000010001BB700FE9FF8F708ED00E09C
:10193000F0B5B049032008630020C1F80801AE48A3
:1019400004228265026C42F004020264AB4A8A6699
:1019500000220A611022C261026822F010020260B5
:101960000322C1F87022C1F8742200224A644FF4A5
:1019700000328261026842F4003202600922C1F83A
:101980000021C1F804211022C1F8D420520482633E
:10199000026A42F4001202620D22C1F8D020C1F89E
:1019A000E0200022C1F8F4204FF00052C263026A26
:1019B00042F0005202620022C1F8F0204FF0805243
:1019C000C263026A42F0805202621022CA670204B5
:1019D0008261026842F0004202601022C1F81421C4
:1019E00020278765026C42F0200202641022C1F8B1
:1019F0001C218022C265026C22F0800202649026C3
:101A0000C1F8FC600204C263026A22F00042026272
:101A10001022C1F8DC20D204C263026A22F4000260
:101A2000026201230B660122CA654A660322C1F8DD
:101A3000D8200522C1F8E42001228A601122CA6060
:101A40000124CC630A640224C1F820411225C1F8A4
:101A500024510C604D600C604D6010248C659C0519
:101A6000C461046844F4800404600124CC630A6403
:101A70001022C1F82C21CA14C265026C42F4006223
:101A800002641022C1F830218A14C265026C42F44B
:101A90008052026440F282224A629A240C62CA6135
:101AA00010224A618761026842F02002026010221F
:101AB0008A6140258561026842F04002026001228D
:101AC0000A67CA6640F20242CA628A621022C1F8FC
:101AD000E82092058263046A44F080640462102462
:101AE000C1F8EC405400C463046A24F0006404624A
:101AF0004E635413C461046824F400540460002449
:101B0000C1F8E841C267026E42F0806202660022BC
:101B1000C1F8E4215A06C267026E42F00072026602
:101B20008A22C1F8F8200822C1F8C820D403C4636F
:101B3000066A46F4802606621026C1F828610E1552
:101B4000C665066C26F4806606640126C1F88060CE
:101B5000C1F88460C1F89060C1F8A060C1F8A460C9
:101B6000C1F8A860C1F8B860C1F8BC60C1F8C06035
:101B7000C1F8C4600026C1F81861C565056C45F060
:101B8000400505640A655504C561056825F480159E
:101B90000560CA641504C561056825F40025056063
:101BA0008A64C461046824F4802404600024C1F8B9
:101BB0000C418265026C42F0080202640022C1F806
:101BC000102110228265026C42F0100202640C485F
:101BD0000C4A0068904204D141F8B83F8B60CB605A
:101BE000F0BD094A9042FBD1812041F8B80F8860CE
:101BF000C860F0BD00C00240008009200200010062
:101C0000C8000010473F1927473F1947FC480021EB
:101C10008180017041704FF001128260C160704795
:101C2000F7491C31002000F0D7BB10B5F44C143438
:101C3000A288402A00D940228020216800F0FDFBC4
:101C4000216801442160A188081AA08010BD10B548
:101C5000EB4C00201434216800F0BEFB21680144E5
:101C60002160A188081AA08010BD002211468020A2
:101C700000F0E3BBE349002000F0AEBB70B5E048E4
:101C8000DF4C1C3004F11404007810F01F000BD05E
:101C9000DB4BDC4D03F11C015A780979012809D08E
:101CA000022813D0002070BDD548001D2060FFF72A
:101CB000BCFF27E042B19878814205D200202880FD
:101CC0002560FFF7B2FF1DE0002070BD01F08F001E
:101CD000010605D500F00F064FF48031B14001E058
:101CE000012181400AB900070ED1986808420BD043
:101CF000D868084201D0012000E00020288025603B
:101D0000FFF793FF012070BD002070BD70B5024643
:101D1000BB4BBB4D1C3319461878498810F01F0087
:101D200005D0012818D0022818D0002070BD012944
:101D300001D0002070BD3AB1012000F0E7FAA88878
:101D400040F00200A8802CE0002000F0DFFAA88814
:101D500020F00200A88024E0002070BD187900F077
:101D60008F00030605D500F00F034FF480349C402C
:101D700001E0012484406B78ABB1030713D0AB685A
:101D8000234210D009B1002070BD2AB100F010FB31
:101D9000E8682043E86004E000F014FBE868A04332
:101DA000E860012070BD002070BD10B594481C3063
:101DB000007810F01F01924800F11C00C07803D099
:101DC00001292FD0002010BD8D4B1433012808D0DD
:101DD00003F1080102288A7807D0032816D00020D2
:101DE00010BD89481860122014E08848002104E0E2
:101DF00004780CB144882044491C8A42F8D1017807
:101E000011B11860408805E0002010BD80481044E2
:101E1000186000789988814200D99880FFF705FF03
:101E2000012010BD002010BD2DE9F05F0027DFF874
:101E3000D0B1734E0BF11C0BB8469BF802004FF06B
:101E400001094FF4803A002868D0704C62E0607855
:101E5000022804D0042840D0052859D13FE06179F8
:101E60009BF80200814235D170702079B07000205B
:101E70006349103101F80080401C0428FAD3012581
:101E8000B16809FA05F0084202D0284600F07CFA51
:101E9000B1680AFA05F0084203D045F0800000F06E
:101EA00073FA6D1C102DEBD34FF001103546B06066
:101EB000C5F80C80012000F02AFAE079400604D52C
:101EC000A88840F00100A88022E0A88820F0010046
:101ED000A8801DE0608804441CE0E77818E0BFB9E2
:101EE000A07800F08F05280604D505F00F000AFA47
:101EF00000F001E009FA05F0B1680143B160204645
:101F000000F01DFA284600F035FA284600F046FA9F
:101F1000207804442078002899D11EE086F80180BA
:101F20000124B16809FA04F0084202D0204600F00A
:101F30002BFAB1680AFA04F0084203D044F080009A
:101F400000F022FA641C102CEBD34FF00110B060AB
:101F5000C6F80C80002000F0DAF99BF802007178D6
:101F6000884202D10120BDE8F09F0020FBE72DE967
:101F7000F84F00270026B246B146DFF884B09BF840
:101F80000100002803D000200090204C72E00020C7
:101F9000BDE8F88F6078022804D004280AD005280C
:101FA00066D11BE060799BF80110884260D06088A0
:101FB00004445FE0A778E6784FF0000910481C3031
:101FC0000179B94254D18078B04251D101200090BA
:101FD0000B48103010F807A0C65549E008481C30DF
:101FE0000179B94244D1A17801F08F085FEA086114
:101FF00010D508F00F014FF480358D400DE0000042
:10200000F4000010301D0010785300008A530000C7
:10201000AB530000012505FA08F58078B04215D1D0
:10202000DBF808002843CBF80800DBF80C00A843D5
:10203000CBF80C00204600F082F9404600F09AF9F7
:10204000404600F0ABF949EA050911E056450FD1C9
:1020500019EA050F0CD1DBF80800A843CBF80800FB
:10206000DBF80C00A843CBF80C00404600F08CF9DC
:1020700020780444207800288CD1009888E72DE946
:10208000F041544F0026A7F108053978A5F1140452
:1020900008281FD2DFE800F01E0477851E1E9994E1
:1020A000FFF7BEFD3878C00900F063F9F888A88012
:1020B0003878C0F3411181BB79780C295ED2DFE812
:1020C00001F0060B5D125D1923272D364253FFF7F1
:1020D000D5FD10B3BDE8F0810020FFF717FEE0B199
:1020E000BDE8F041C1E50120FFF710FEA8B1BDE851
:1020F000F041BAE510F01F0F40D1B87840F08000F1
:102100002070BDE8F041B0E5FFF74FFE28B1E1E7F0
:10211000002000F04DF9AE80DCE72FE010F01F0F3B
:102120002CD12C481B382860BDE8F0417DE510F02B
:102130001F0F23D1FFF778FE00B3FFF796FDBDE830
:10214000F04100F07DBA00F01F00012816D1607840
:10215000A0B13879A178884210D21E490C390844C0
:102160002860BDE8F04160E500F01F00012805D1BE
:10217000FFF7FDFE10B1BDE8F04176E5802000F0EC
:1021800017F9AE80A6E7080608D4A8880028A1D0D1
:10219000FFF75DFDA8880028F0D09BE7BDE8F0417F
:1021A00068E5080602D5BDE8F0413EE52078010665
:1021B00090D500F07F002070BDE8F04100F054B8E9
:1021C000BDE8F041802000F0FDB8BDE8F0410020FE
:1021D00000F0F8B81001001001460807C00E09060B
:1021E00000D5401C7047DB491022C1F80822C1F815
:1021F0001002D1F80002C006FBD57047D54A102363
:10220000C2F80832C2F81002D2F80002C006FBD5AC
:10221000C2F80832C2F81012D2F80002C006FBD58C
:102220007047CC493022C1F80822C1F81002D1F819
:1022300000028006FBD5D1F81402704710B50446A1
:10224000002C01D0012100E000214FF4807040EA11
:102250000141C148FFF7D2FFC0484FF480210CB1C3
:10226000816310BDC16310BD30B540F080014FF4F3
:10227000807040EA0141BA4D0C462846FFF7BEFF88
:1022800021462846BDE83040B8E7B6480021016045
:1022900040214160012202604160A0F51270D0F837
:1022A0000012C905FBD500F501704FF0FF31416305
:1022B000016341600C210160704730B5AA4C1A23BC
:1022C0002360211D0A6833EA0200FBD1A7480122DE
:1022D00042678267A64D00222A608A22C0F8F82051
:1022E00023600A6833EA0200FBD1A2494FF08070F4
:1022F000C1F8FC01A04B20221A70C867FFF7C5FF88
:10230000BDE830400020AFE770477047704710B518
:10231000002801D0012000E000204FF4807444EA3E
:1023200000419648FFF76AFF8A480321C0F844122B
:10233000D0F80012C905FBD5C0F8084210BD10B591
:1023400002469078FFF748FF8649091F0B68012471
:10235000844023430B60486090888860A1F5117128
:10236000D1F80002C005FBD54FF48070C1F8080217
:1023700010BD704700B5FFF72FFF81495DF804EBF2
:1023800041EA0040891339E700B5FFF725FF7C4992
:102390005DF804EB41EA00407A492FE700B5FFF70A
:1023A0001BFF77495DF804EB41EA0040891325E7FC
:1023B00000B5FFF711FF72495DF804EB41EA0040F8
:1023C00071491BE700B5FFF707FF6D495DF804EBA6
:1023D00041EA0040891311E770B506465D4B06F0EF
:1023E0000F00012202EB8000C3F82802D3F820027C
:1023F0000205FBD5C0F309050022EC1C04E0D3F86C
:10240000180241F8040B521CB2EB940FF7D30020D2
:10241000C3F8280241F24820F040C0070BD13046F3
:10242000FFF7DAFE4FF4A06141EA0040FFF7DBFE60
:102430005648FFF7D8FE284670BD70B51646454D84
:1024400000F00F02022303EB8202C5F82822C5F830
:1024500024620023F41C04E051F8042BC5F81C226C
:102460005B1CB3EB940FF7D30021C5F82812FFF7DC
:10247000B3FE4FF4A06141EA0040FFF7B4FE4448C8
:10248000FFF7B1FE304670BD2DE9F041314FD7F86E
:102490000032C7F80832180725D52F48FFF7A3FEEA
:1024A0003C48FFF7BEFEC10605D5FFF7EEFEBDE8CE
:1024B000F04100F0B6B8810705D5BDE8F04100F065
:1024C000010000F0A8B801070DD5400705D5FFF7BA
:1024D0001BFFBDE8F04100F0ABB8FFF716FFBDE809
:1024E000F04100F0ACB8580721D54FF001082A4E52
:1024F00019E00024D7F8300208FA04F528420FD07A
:102500006008C7F83852D7F800128906FBD5D7F80B
:102510001412E2070DD056F8201009B103208847A5
:10252000641C202CE6D3D7F830020028E1D1BDE8A6
:10253000F0813CB9490705D5316819B131680120EE
:102540008847EDE756F820100029E9D00220884797
:10255000E6E7000000C008200005FE00008009201A
:102560000005D00048C20820F4CF082000C0024077
:1025700010C1082084E000E018E400E00005D80065
:102580000005400000012000000101000005F200EC
:102590000005FA000002FE001C54000070B52D4C2E
:1025A000607800282DD000252B4E012810D002285D
:1025B0000DD1B0686168401A284988421BD3284869
:1025C000406B400017D50120FFF738FE657070BDE5
:1025D000B0686168401A23498842F8D30020FFF7A9
:1025E0002DFEB0686060022060702570BDE870400C
:1025F0000C20FEF755BF2570BDE870400C20FEF79B
:102600004FBF20780028E2D101202070BDE8704043
:102610000D20FEF745BF002802D10E490120487069
:10262000704710B5FFF7F2FA0A490020487010BD54
:102630000848012141700849896841607047704726
:102640007047022803D0032803D1FEF74CBDFEF7E4
:1026500069BD70471801001000000940A086010004
:102660000080092040420F0019480621016107211E
:10267000016000214161416202214160C168C906D7
:10268000FCD400E08168C1684907FBD40020704792
:102690000F498860C868C006FCD48868704700B5D8
:1026A00002460B4603E012F8010BFFF7F1FF5B1E39
:1026B000581CF8D100BD00B502460B4604E00020CE
:1026C000FFF7E6FF02F8010B5B1E581CF7D100BDB7
:1026D0000000034070B5044600BF00BF00BF00BF4C
:1026E00000BF00BF00BF00BF00BF00BF00BF00BFF2
:1026F00000BF00BF00BF00BF00BF00BF00BF00BFE2
:1027000000BF00BF00BF00BF00BF00BF00BF00BFD1
:1027100000BF00BF00BF00BF4026FE4DEE61052098
:10272000FFF7B6FF0020FFF7B3FF2070AE6100BFD8
:1027300000BF00BF00BF00BF00BF00BF00BF00BFA1
:1027400000BF00BF00BF00BF00BF00BF00BF00BF91
:1027500000BF00BF00BF00BF00BF00BF00BF00BF81
:1027600000BF00BF00BF00BF00BF00BF00BF207898
:1027700000F0010070BD2DE9F04106460F46E64C21
:10278000A56806E0A068401BB04202D30120BDE866
:10279000F0813846FFF79EFF0028F3D1F7E72DE9D7
:1027A000F0478146DD4E4FF0807740243068D94DA8
:1027B000B84249D100BF00BF00BF00BF00BF00BF8B
:1027C00000BF00BF00BF00BF00BF00BF00BF00BF11
:1027D00000BF00BF00BF00BF00BF00BF00BF00BF01
:1027E00000BF00BF00BF00BF00BF00BF00BF00BFF1
:1027F00000BF00BFEC611520FFF74AFF0020FFF784
:1028000047FF00F0FF08AC6100BF00BF00BF00BF82
:1028100000BF00BF00BF00BF00BF00BF00BF00BFC0
:1028200000BF00BF00BF00BF00BF00BF00BF00BFB0
:1028300000BF00BF00BF00BF00BF00BF00BF00BFA0
:1028400000BF00BF00BF00BF00BF00BF00BF00BF90
:1028500000BF00BF00BF00BF00BF00BF00BF00BF80
:1028600000BF00BF00BF00BF00BF00BF00BF00BF70
:1028700000BF00BF00BF00BF00BF00BF00BF00BF60
:1028800000BF00BF00BF00BFEC610620FFF700FFE4
:10289000AC6100BF00BF00BF00BF00BF00BF00BFF2
:1028A00000BF00BF00BF00BF00BF00BF00BF00BF30
:1028B00000BF00BF00BF00BF00BF00BF00BF00BF20
:1028C00000BF00BF00BF00BF00BF00BF00BF00BF10
:1028D00000BF00BF00BF00BF00BF00BF00BF00BF00
:1028E00000BF00BF00BF00BF00BF00BF00BF00BFF0
:1028F00000BF00BF00BF00BF00BF00BF00BF00BFE0
:1029000000BF00BF00BF00BF00BF00BF00BF00BFCF
:1029100000BFEC610120FFF7BBFE4FEA8900FFF723
:10292000B7FE3068B84202D14046FFF7B1FEAC6155
:1029300000BF00BF00BF00BF00BF00BF00BF00BF9F
:1029400000BF00BF00BF00BF00BF00BF00BF00BF8F
:1029500000BF00BF00BF00BF00BF00BF00BF00BF7F
:1029600000BF00BF00BF00BF00BF00BF00BF00BF6F
:10297000BDE8F0872DE9FC5F044688466946684853
:10298000FFF7F9FE674D684E684F4FF0820A40B17D
:10299000C5F800A022203060784638608220BDE86B
:1029A000FC9F03208DF8040020098DF8050020010C
:1029B0008DF806004FF000098DF8079000BF00BFAA
:1029C00000BF00BF00BF00BF00BF00BF00BF00BF0F
:1029D00000BF00BF00BF00BF00BF00BF00BF00BFFF
:1029E00000BF00BF00BF00BF00BF00BF00BF00BFEF
:1029F00000BF00BF00BF00BF00BF00BF4020DFF826
:102A000014B1CBF81C00042101A8FFF748FE0024F4
:102A10000020FFF73DFEC0B2009018F80410884275
:102A200007D0C5F800A022203060784638608220A8
:102A3000B5E7641CB4F5805FEAD34020CBF81800FA
:102A400000BF00BF00BF00BF00BF00BF00BF00BF8E
:102A500000BF00BF00BF00BF00BF00BF00BF00BF7E
:102A600000BF00BF00BF00BF00BF00BF00BF00BF6E
:102A700000BF00BF00BF00BF00BF00BF00BF00BF5E
:102A8000C5F80090C6F8009078463860002086E7C8
:102A90002DE9F8430025009500BF00BF00BF00BF2F
:102AA00000BF00BF00BF00BF00BF00BF00BF00BF2E
:102AB00000BF00BF00BF00BF00BF00BF00BF00BF1E
:102AC00000BF00BF00BF00BF00BF00BF00BF00BF0E
:102AD00000BF00BF00BF00BF40260E4FFE619F2019
:102AE000FFF7D6FD0020FFF7D3FDC4B28DF80040FC
:102AF0000020FFF7CDFD00F0FF098DF801900020C8
:102B0000FFF7C6FDC0B28DF80200BE6100BF00BF76
:102B100000BF0DE0008009200000094020010010E6
:102B2000A0860100700000107400001078000010F2
:102B300000BF00BF00BF00BF00BF00BF00BF00BF9D
:102B400000BF00BF00BF00BF00BF00BF00BF00BF8D
:102B500000BF00BF00BF00BF00BF00BF00BF00BF7D
:102B600000BF00BF00BF00BF00BFFC4EFC4FDFF83E
:102B7000F483C22C02D1B9F1200F09D08220306039
:102B8000212038607846C8F800008220BDE8F8832C
:102B9000F549142810D0152812D0162814D018285A
:102BA00016D00D600020FFF7FAFD35603D607846D5
:102BB000C8F800000020E9E74FF480100860F1E752
:102BC0004FF400100860EDE74FF480000860E9E77B
:102BD0004FF080700860E5E72DE9F34FC3B005467C
:102BE0000024DFF87883DFF87893DFF878A30027F4
:102BF00042A9DE48FFF7BFFD60B18220C8F800009F
:102C00002120C9F800007846CAF80000822045B0AB
:102C1000BDE8F08F00F00DFB02208DF804002809BC
:102C20008DF8050004EB05108DF806008DF807708F
:102C300044984FF4807200EB042102A8FDF738FBA2
:102C400000BF00BF00BF00BF00BF00BF00BF00BF8C
:102C500000BF00BF00BF00BF00BF00BF00BF00BF7C
:102C600000BF00BF00BF00BF00BF00BF00BF00BF6C
:102C700000BF00BF00BF00BF00BF00BF00BF00BF5C
:102C80004026DFF8ECB2CBF81C604FF4827101A84B
:102C9000FFF705FDCBF8186000BF00BF00BF00BF05
:102CA00000BF00BF00BF00BF00BF00BF00BF00BF2C
:102CB00000BF00BF00BF00BF00BF00BF00BF00BF1C
:102CC00000BF00BF00BF00BF00BF00BF00BF00BF0C
:102CD00000BF00BF00BF00BF641CE4B2102C87D34C
:102CE00042A9A248FFF747FD50B18220C8F8000072
:102CF0002120C9F800007846CAF80000822086E743
:102D000000F0E0FAC8F80070C9F800707846CAF818
:102D1000000000207BE72DE9FF5F8A46174600256B
:102D2000DFF83882DFF838B2002F12D04FF4805429
:102D3000014622466846FDF7B1FADDE90001CDE91A
:102D40000201204602F04AF881465FEA09000DD0F0
:102D500017E08620C8F800000920CBF8000079466B
:102D600080480160862004B0BDE8F09F8220C8F84A
:102D700000002220CBF8000079467A4801608220CA
:102D8000F1E700247E1B0398C0F58050B04200D2CA
:102D90000646B6F5805F0AD04946029800F021FD4C
:102DA00028B1484601F0F2FFD8F80000DBE70398AD
:102DB0000AEB050148443246FDF77AFA029800F022
:102DC00096FC28B1484601F0E1FFD8F80000CAE7B8
:102DD00049460298FFF700FF28B1484601F0D6FFA8
:102DE000D8F80000BFE749460298FFF7C3FD48B195
:102DF000641CE4B2032C06D3484601F0C7FFD8F8A0
:102E00000000B0E70024002CD8D135440298401CC3
:102E1000029000200390BD42B3D3484601F0B6FFB4
:102E20000020C8F80000CBF8000079464D4801604A
:102E3000002098E72DE9F04F89B00D46DDF8489065
:102E400092461F460024DFF81481B9F1000F4DD0DF
:102E50004FF480560146324601A8FDF71FFADDE91E
:102E60000101CDE905013246691C01A8FDF716FAFA
:102E7000DDE90101CDE903013246514601A8FDF724
:102E80000DFADDE90101CDE90701A346A9EB04052F
:102E90000898C0F58050A84200D20546089838B17D
:102EA00005990798884258D1069908988842FAD11E
:102EB0004FF4805001F092FF0646300021D0059972
:102EC000079888427DD10699089888427FD1DDE92C
:102ED00007020003314600F04AFB00061CD53046CD
:102EE00001F054FFD8F8000009B091E68620C8F838
:102EF00000001B480921016079461A4801608620BC
:102F0000F2E78220C8F800001548222101607946C6
:102F1000144801608220E7E703990798884211D19D
:102F2000DDE9031000EB01300499C1F58052314412
:102F300000F01DFB000605D5304601F027FFD8F84C
:102F40000000D1E7079800F0D2FB000612D530460A
:102F500001F01CFFD8F80000C6E781E07000001007
:102F6000740000107800001020010010A0860100FD
:102F7000008009200898391930442A46FDF798F94D
:102F80000898314642190798000301F0A0FA00069C
:102F900005D5304601F0FAFED8F80000A4E7039901
:102FA0000798884258D1DDE9031000EB01300499FD
:102FB000C1F58052314401F08AFA00064CD5304602
:102FC00000E004E001F0E2FED8F800008CE703998D
:102FD0000798884211D1DDE9031000EB0130049914
:102FE000C1F58052314600F0C2FA000605D53046E0
:102FF00001F0CCFED8F8000076E7079800F077FBE8
:10300000000605D5304601F0C1FED8F800006BE798
:1030100039190AEB04002A4601F059FA000605D5D1
:10302000304601F0B3FED8F800005DE70399079839
:10303000884211D1DDE9031000EB01300499C1F59C
:103040008052314601F043FA000605D5304601F0C2
:103050009DFED8F8000047E7304601F097FE0AE0F1
:1030600039190AEB04002A4601F031FA000602D5AC
:10307000D8F8000038E72C440798401C0790CDF89A
:1030800020B04C45FFF402AFC8F800B03248C0F899
:1030900000B0794631480160002025E730480068DB
:1030A00070474FF4805070472DE9F04786B00546D1
:1030B0000E460024DFF8AC80DFF89C90DFF89CA07F
:1030C000002E2ED04FF480573A4629466846FDF729
:1030D000E5F8DDE90001CDE902013A4629466846F6
:1030E000FDF7DCF8DDE90001CDE904010027351B1F
:1030F0000598C0F58050A84200D20546059838B121
:1031000002990498884217D103990598884213D1EF
:10311000049800F0ECFA00060ED5D8F8000006B0CE
:1031200026E48620C8F800000920C9F80000784687
:10313000CAF800008620F2E72C440498401C049052
:103140000597B442D3D3C8F80070C9F80070784628
:10315000CAF800000020E2E77400001078000010B8
:10316000200100107000001070B5044600BF00BFC1
:1031700000BF00BF00BF00BF00BF00BF00BF00BF57
:1031800000BF00BF00BF00BF00BF00BF00BF00BF47
:1031900000BF00BF00BF00BF00BF00BF00BF00BF37
:1031A00000BF00BF00BF00BF00BF00BF4026FD4DF5
:1031B000EE610520FFF76CFA0020FFF769FA207036
:1031C000AE6100BF00BF00BF00BF00BF00BF00BFB7
:1031D00000BF00BF00BF00BF00BF00BF00BF00BFF7
:1031E00000BF00BF00BF00BF00BF00BF00BF00BFE7
:1031F00000BF00BF00BF00BF00BF00BF00BF00BFD7
:1032000000BF207800F0010070BD2DE9F0410646B6
:103210000F46E54CA56806E0A068401BB04202D30B
:103220000120BDE8F0813846FFF79EFF0028F3D16A
:10323000F7E770B500BF00BF00BF00BF00BF00BF11
:1032400000BF00BF00BF00BF00BF00BF00BF00BF86
:1032500000BF00BF00BF00BF00BF00BF00BF00BF76
:1032600000BF00BF00BF00BF00BF00BF00BF00BF66
:1032700000BF00BF4025CB4CE5610620FFF708FAF0
:10328000A56100BF00BF00BF00BF00BF00BF00BFFF
:1032900000BF00BF00BF00BF00BF00BF00BF00BF36
:1032A00000BF00BF00BF00BF00BF00BF00BF00BF26
:1032B00000BF00BF00BF00BF00BF00BF00BF00BF16
:1032C00000BF70BD70B500BF00BF00BF00BF00BF32
:1032D00000BF00BF00BF00BF00BF00BF00BF00BFF6
:1032E00000BF00BF00BF00BF00BF00BF00BF00BFE6
:1032F00000BF00BF00BF00BF00BF00BF00BF00BFD6
:1033000000BF00BF00BF4025A64CE5610420FFF7C9
:10331000BFF9A56100BF00BF00BF00BF00BF00BF75
:1033200000BF00BF00BF00BF00BF00BF00BF00BFA5
:1033300000BF00BF00BF00BF00BF00BF00BF00BF95
:1033400000BF00BF00BF00BF00BF00BF00BF00BF85
:1033500000BF00BF70BD70B5064600BF00BF00BF14
:1033600000BF00BF00BF00BF00BF00BF00BF00BF65
:1033700000BF00BF00BF00BF00BF00BF00BF00BF55
:1033800000BF00BF00BF00BF00BF00BF00BF00BF45
:1033900000BF00BF00BF00BF00BF4024814DEC61F3
:1033A0005020FFF775F9AC6100BF00BF00BF00BF40
:1033B00000BF00BF00BF00BF00BF00BF00BF00BF15
:1033C00000BF00BF00BF00BF00BF00BF00BF00BF05
:1033D00000BF00BF00BF00BF00BF00BF00BF00BFF5
:1033E00000BF00BF00BF00BF00BF00BF00BF00BFE5
:1033F00000BF00BF00BF00BF00BF00BF00BF00BFD5
:1034000000BF00BF00BF00BF00BF00BF00BF00BFC4
:1034100000BF00BF00BF00BF00BF00BF00BF00BFB4
:1034200000BF00BF00BF00BFEC610120FFF730F913
:10343000B000FFF72DF9AC6100BF00BF00BF00BFB7
:1034400000BF00BF00BF00BF00BF00BF00BF00BF84
:1034500000BF00BF00BF00BF00BF00BF00BF00BF74
:1034600000BF00BF00BF00BF00BF00BF00BF00BF64
:1034700000BF00BF00BF00BF70BD2DE9FE43044682
:103480000D4602A94948FFF7C0FE494E494FDFF8F3
:10349000288148B182203060222038607846C8F800
:1034A00000008220BDE8FE839DF80800800701D45B
:1034B000FFF7BFFE02208DF80000200C8DF8010000
:1034C000200A8DF802008DF803408DF8045000BFEB
:1034D00000BF00BF00BF00BF00BF00BF00BF00BFF4
:1034E00000BF00BF00BF00BF00BF00BF00BF00BFE4
:1034F00000BF00BF00BF00BF00BF00BF00BF00BFD4
:1035000000BF00BF00BF00BF00BF00BF00BF40251D
:10351000244CE56105216846FFF7C1F8A56100BFAD
:1035200000BF00BF00BF00BF00BF00BF00BF00BFA3
:1035300000BF00BF00BF00BF00BF00BF00BF00BF93
:1035400000BF00BF00BF00BF00BF00BF00BF00BF83
:1035500000BF00BF00BF00BF00BF00BF00BF002012
:10356000306038607846C8F8000000209AE72DE9FE
:10357000FC5F04468A4691460D4D0E4E0E4F4FF0AD
:103580000008B9F1000F19D001A90848FFF73DFE66
:10359000E0B18220286021203060784638608220A7
:1035A000BDE8FC9F0080092000000940A0860100C2
:1035B000700000107400001078000010C5F8008042
:1035C000C6F80080784638600020E9E703208DF8CF
:1035D0000000200C8DF80100200A8DF802008DF803
:1035E000034000BF00BF00BF00BF00BF00BF00BF5F
:1035F00000BF00BF00BF00BF00BF00BF00BF00BFD3
:1036000000BF00BF00BF00BF00BF00BF00BF00BFC2
:1036100000BF00BF00BF00BF00BF00BF00BF00BFB2
:1036200000BF4024DFF86CB4CBF81C40042168468E
:10363000FFF735F849465046FFF73DF8CBF81840FC
:1036400000BF00BF00BF00BF00BF00BF00BF00BF82
:1036500000BF00BF00BF00BF00BF00BF00BF00BF72
:1036600000BF00BF00BF00BF00BF00BF00BF00BF62
:1036700000BF00BF00BF00BF00BF00BF00BF00BF52
:10368000C5F80080C6F8008078463860002087E7DB
:103690002DE9F05F80460D461646FF4FDFF8FCA38C
:1036A000DFF8FCB34FF00009002E01D0002413E036
:1036B000C7F80090CAF800907846CBF800000020C8
:1036C000BDE8F09F295D08EB0400FFF7D6FE000679
:1036D00001D53868F4E7641CB442F3D3C7F800900E
:1036E000CAF800907846CBF800000020E8E72DE902
:1036F000FC47044601A9EB48FFF787FDE64FDFF8DA
:103700009C83DFF89C9350B1822038602220C8F857
:1037100000007846C9F800008220BDE8FC879DF8CB
:103720000400800701D4FFF784FD20208DF80000FD
:1037300020098DF8010020018DF8020000248DF889
:10374000034000BF00BF00BF00BF00BF00BF00BFFD
:1037500000BF00BF00BF00BF00BF00BF00BF00BF71
:1037600000BF00BF00BF00BF00BF00BF00BF00BF61
:1037700000BF00BF00BF00BF00BF00BF00BF00BF51
:1037800000BF4026C34DEE6104216846FEF787FF67
:10379000AE6100BF00BF00BF00BF00BF00BF00BFE1
:1037A00000BF00BF00BF00BF00BF00BF00BF00BF21
:1037B00000BF00BF00BF00BF00BF00BF00BF00BF11
:1037C00000BF00BF00BF00BF00BF00BF00BF00BF01
:1037D00000BF3C60C8F800407846C9F800000020EF
:1037E0009BE72DE9FC4704468A4601A9AD48FFF74F
:1037F0000CFDA94FDFF8A482DFF8A49248B1822023
:1038000038602220C8F800007846C9F800008220FD
:1038100083E703208DF8000020098DF801002001C6
:103820008DF8020000248DF8034000BF00BF00BFE8
:1038300000BF00BF00BF00BF00BF00BF00BF00BF90
:1038400000BF00BF00BF00BF00BF00BF00BF00BF80
:1038500000BF00BF00BF00BF00BF00BF00BF00BF70
:1038600000BF00BF00BF00BF00BF4025894EF5610B
:1038700004216846FEF713FFA9015046FEF71BFF1F
:10388000B56100BF00BF00BF00BF00BF00BF00BFE9
:1038900000BF00BF00BF00BF00BF00BF00BF00BF30
:1038A00000BF00BF00BF00BF00BF00BF00BF00BF20
:1038B00000BF00BF00BF00BF00BF00BF00BF00BF10
:1038C00000BF3C60C8F800407846C9F800000020FE
:1038D00023E72DE9FC5F04468B4601A97148FFF7F9
:1038E00094FC6D4FDFF8B481DFF8B4914FF0820A99
:1038F00048B1C7F800A02120C8F800007846C9F8F0
:10390000000082204CE69DF80400800701D4FFF7F8
:1039100090FCAD208DF8000020098DF801002001F9
:103920008DF8020000208DF8030000BF00BF00BF2B
:1039300000BF00BF00BF00BF00BF00BF00BF00BF8F
:1039400000BF00BF00BF00BF00BF00BF00BF00BF7F
:1039500000BF00BF00BF00BF00BF00BF00BF00BF6F
:1039600000BF00BF00BF00BF00BF4025494EF5614A
:1039700004216846FEF793FE02215846FEF78FFEAB
:10398000B56100BF00BF00BF00BF00BF00BF00BFE8
:1039900000BF00BF00BF00BF00BF00BF00BF00BF2F
:1039A00000BF00BF00BF00BF00BF00BF00BF00BF1F
:1039B00000BF00BF00BF00BF00BF00BF00BF00BF0F
:1039C00000BF022401A93748FFF71FFC48B1C7F820
:1039D00000A02220C8F800007846C9F80000822024
:1039E000DEE500BF00BF00BF00BF00BF00BF00BFDB
:1039F00000BF00BF00BF00BF00BF00BF00BF00BFCF
:103A000000BF00BF00BF00BF00BF00BF00BF00BFBE
:103A100000BF00BF00BF00BF00BF00BF00BF00BFAE
:103A200000BFF561AD20FEF733FE0BEB0400022171
:103A3000FEF735FEB56100BF00BF00BF00BF00BF8D
:103A400000BF00BF00BF00BF00BF00BF00BF00BF7E
:103A500000BF00BF00BF00BF00BF00BF00BF00BF6E
:103A600000BF00BF00BF00BF00BF00BF00BF00BF5E
:103A700000BF00BF00BFA41CA4B2B4F5805FA1D3F7
:103A800001A90848FFF7C1FBA8B1C7F800A0212091
:103A90000AE000000080092070000010740000108F
:103AA00078000010A0860100C8F800007846C9F828
:103AB0000000822074E5FFF705FC00203860C8F89C
:103AC00000007846C9F80000002069E570B5FD4D9A
:103AD000FD4EFE4C002A05D0FFF749FD000609D532
:103AE000206870BD862020600920286078463060FC
:103AF000862070BD0020206028607846306000205D
:103B000070BD2DE9FF5F894616460024DFF8BC83AF
:103B1000DFF8B0B3002E27D04FF4805501462A4677
:103B20006846FCF7BBFBDDE90001CDE90201284650
:103B300001F054F90746380021D0A246351B0398FE
:103B4000C0F58050A84200D20546B5F5805F21D06F
:103B500039460298FFF745FEE0B1384601F016F904
:103B6000D8F8000004B0ABE58620C8F800000920B2
:103B7000CBF800007946D44801608620F2E7822025
:103B8000C8F800002220CBF800007946CE4801603A
:103B90008220E7E70298FFF7AAFD28B1384601F036
:103BA000F5F8D8F80000DDE7039809EB0401384484
:103BB0002A46FCF77DFB2C4439460298FFF789FE24
:103BC00028B1384601F0E2F8D8F80000CAE70298B8
:103BD000401C0290CDF80CA0B442AFD3384601F09F
:103BE000D5F8C8F800A0CBF800A07946B648016027
:103BF0000020B7E72DE9F04F89B00D46DDF8489079
:103C000092461F460024DFF8C482B9F1000F4ED05F
:103C10004FF480560146324601A8FCF73FFBDDE930
:103C20000101CDE905013246691C01A8FCF736FB0C
:103C3000DDE90101CDE903013246514601A8FCF757
:103C40002DFBDDE90101CDE90701A346A9EB040540
:103C50000898C0F58050A84200D20546089838B1AF
:103C60000599079888426ED1069908988842FAD13A
:103C70004FF4805001F0B2F80646300022D005998A
:103C80000798884277D106990898884273D1DDE970
:103C9000070200033146FFF76AFC00061DD53046D7
:103CA00001F074F8D8F8000009B0BDE8F08F862064
:103CB000C8F8000083480921016079468248016004
:103CC0008620F1E78220C8F800007E4822210160AA
:103CD00079467D4801608220E6E70399079888428B
:103CE00011D1DDE9031000EB01300499C1F58052D8
:103CF0003144FFF73CFC000605D5304601F046F89C
:103D0000D8F80000D0E70798FFF7F1FC000605D5CA
:103D1000304601F03BF8D8F80000C5E7089839199B
:103D200030442A46FCF7C4FA0898314642190798ED
:103D30000003FFF7ADFC000606D5304601F026F87B
:103D4000D8F80000B0E75FE003990798884257D1A0
:103D5000DDE9031000EB01300499C1F580523144D4
:103D6000FFF796FC00064BD5304601F00FF8D8F867
:103D7000000099E7FFE703990798884211D1DDE930
:103D8000031000EB01300499C1F580523146FFF772
:103D9000EEFB000605D5304600F0F8FFD8F800002D
:103DA00082E70798FFF7A3FC000605D5304600F030
:103DB000EDFFD8F8000077E739190AEB04002A462E
:103DC000FFF766FC000605D5304600F0DFFFD8F8A7
:103DD000000069E703990798884211D1DDE90310D3
:103DE00000EB01300499C1F580523146FFF750FCD9
:103DF000000605D5304600F0C9FFD8F8000053E7AB
:103E0000304600F0C3FF0AE039190AEB04002A46E5
:103E1000FFF73EFC000602D5D8F8000044E72C442A
:103E20000798401C0790CDF820B04C45FFF40EAF2A
:103E3000C8F800B02348C0F800B0794622480160B5
:103E4000002031E72DE9F8430026009600BF00BFAF
:103E500000BF00BF00BF00BF00BF00BF00BF00BF6A
:103E600000BF00BF00BF00BF00BF00BF00BF00BF5A
:103E700000BF00BF00BF00BF00BF00BF00BF00BF4A
:103E800000BF00BF00BF00BF00BF00BF4027DFF87A
:103E90004080C8F81C709F20FEF7FAFB0020FEF758
:103EA000F7FBC5B28DF800500020FEF7F1FBC4B25D
:103EB0008DF801400020FEF7EBFBC0B28DF8020048
:103EC00008E000007400001078000010700000107E
:103ED00000800920C8F8187000BF00BF00BF00BFF5
:103EE00000BF00BF00BF00BF00BF00BF00BF00BFDA
:103EF00000BF00BF00BF00BF00BF00BF00BF00BFCA
:103F000000BF00BF00BF00BF00BF00BF00BF00BFB9
:103F100000BF00BF00BF00BF864FDFF81C82DFF884
:103F20001C92BF2D03D1252C0CD0262C0AD0822028
:103F300038602120C8F800007846C9F800008220C7
:103F4000BDE8F8837E49412811D04FF48002422811
:103F500013D04A280FD00E600020FFF7FCF93E6016
:103F6000C8F800607846C9F800000020E8E74FF480
:103F700000100860F0E70A60EEE70A60ECE72DE960
:103F8000F84F69466F48FFF740F96A4C6A4D6B4E2F
:103F90004FF082094FF0220A40B1C4F80090C5F8F2
:103FA00000A0784630608220BDE8F88F9DF80000C0
:103FB000800701D4FFF73DF900BF00BF00BF00BF7D
:103FC00000BF00BF00BF00BF00BF00BF00BF00BFF9
:103FD00000BF00BF00BF00BF00BF00BF00BF00BFE9
:103FE00000BF00BF00BF00BF00BF00BF00BF00BFD9
:103FF00000BF00BF00BF00BF534F4FF04008C7F8DD
:104000001C806020FEF744FBC7F8188000BF00BF8B
:1040100000BF00BF00BF00BF00BF00BF00BF00BFA8
:1040200000BF00BF00BF00BF00BF00BF00BF00BF98
:1040300000BF00BF00BF00BF00BF00BF00BF00BF88
:1040400000BF00BF00BF00BF00BF00BF69463F48C0
:10405000FFF7DBF838B1C4F80090C5F800A0784647
:1040600030608220A0E70020206028607846306021
:10407000002099E73248006870474FF4805070473D
:104080002DE9F04786B005460E460024DFF8A480EF
:10409000DFF8A490DFF8A4A0002E2FD04FF48057B3
:1040A0003A4629466846FCF7F9F8DDE90001CDE912
:1040B00002013A4629466846FCF7F0F8DDE90001BE
:1040C000CDE904010027351B0598C0F58050A842B2
:1040D00000D20546059838B102990498884218D153
:1040E00003990598884214D10498FFF700FB000655
:1040F0000FD5D8F8000006B0BDE8F0878620C8F8D4
:1041000000000920C9F800007846CAF8000086209F
:10411000F1E72C440498401C04900597B442D2D394
:10412000C8F80070C9F800707846CAF8000000208E
:10413000E1E700007000001074000010780000102B
:1041400024010010A08601000080092020A10700A2
:1041500070B5044600BF00BF00BF00BF00BF00BF76
:1041600000BF00BF00BF00BF00BF00BF00BF00BF57
:1041700000BF00BF00BF00BF00BF00BF00BF00BF47
:1041800000BF00BF00BF00BF00BF00BF00BF00BF37
:1041900000BF00BF4026FE4DEE610520FEF778FA15
:1041A0000020FEF775FA2070AE6100BF00BF00BFAF
:1041B00000BF00BF00BF00BF00BF00BF00BF00BF07
:1041C00000BF00BF00BF00BF00BF00BF00BF00BFF7
:1041D00000BF00BF00BF00BF00BF00BF00BF00BFE7
:1041E00000BF00BF00BF00BF00BF207800F001008B
:1041F00070BD2DE9F04106460F46E64CA56806E085
:10420000A068401BB04202D30120BDE8F0813846CF
:10421000FFF79EFF0028F3D1F7E72DE9FF4703A939
:10422000DD48FFF7E6FFDD4FDFF87483DFF87493B6
:1042300058B1822038602120C8F800007846C9F8BB
:104240000000822004B0BDE8F0879DF80C008007D4
:1042500001D4FEF7EEFF42208DF800000024CDF8D7
:104260000140CDF80540ADF8094000BF00BF00BFD8
:1042700000BF00BF00BF00BF00BF00BF00BF00BF46
:1042800000BF00BF00BF00BF00BF00BF00BF00BF36
:1042900000BF00BF00BF00BF00BF00BF00BF00BF26
:1042A00000BF00BF00BF00BF00BF4026B84DEE6199
:1042B0000B216846FEF7F3F9AE6100BF00BF00BFF7
:1042C00000BF00BF00BF00BF00BF00BF00BF00BFF6
:1042D00000BF00BF00BF00BF00BF00BF00BF00BFE6
:1042E00000BF00BF00BF00BF00BF00BF00BF00BFD6
:1042F00000BF00BF00BF00BF00BF3C60C8F8004067
:104300007846C9F8000000209CE72DE9F34F85B0FE
:10431000044604A9A048FFF76CFFA04DA04EA14F92
:104320004FF0820A48B1C5F800A0212030607846DD
:104330003860822007B0BDE8F08FFEF77AFF422098
:104340008DF804004FF0000BCDF805B0CDF809B0A2
:10435000ADF80DB000BF00BF00BF00BF00BF00BF81
:1043600000BF00BF00BF00BF00BF00BF00BF00BF55
:1043700000BF00BF00BF00BF00BF00BF00BF00BF45
:1043800000BF00BF00BF00BF00BF00BF00BF00BF35
:1043900000BF00BFDFF8F8814FF04009C8F81C905B
:1043A0000B2101A8FEF77BF9C8F8189000BF00BFE9
:1043B00000BF00BF00BF00BF00BF00BF00BF00BF05
:1043C00000BF00BF00BF00BF00BF00BF00BF00BFF5
:1043D00000BF00BF00BF00BF00BF00BF00BF00BFE5
:1043E00000BF00BF00BF00BF00BF00BF04A96A48F4
:1043F000FFF7FFFE38B1C5F800A0222030607846F4
:104400003860822096E79DF81000800701D4FEF7FF
:1044100010FF02208DF80400200C8DF80500200A02
:104420008DF806008DF8074006988DF8080000BF4B
:1044300000BF00BF00BF00BF00BF00BF00BF00BF84
:1044400000BF00BF00BF00BF00BF00BF00BF00BF74
:1044500000BF00BF00BF00BF00BF00BF00BF00BF64
:1044600000BF00BF00BF00BF00BF00BF00BFC8F853
:104470001C90052101A8FEF712F9C8F8189000BF9A
:1044800000BF00BF00BF00BF00BF00BF00BF00BF34
:1044900000BF00BF00BF00BF00BF00BF00BF00BF24
:1044A00000BF00BF00BF00BF00BF00BF00BF00BF14
:1044B00000BF00BF00BF00BF00BF00BF00BFC5F806
:1044C00000B0C6F800B078463860002032E72DE929
:1044D000F05F80460D461646304FDFF8C4A0DFF887
:1044E000C4B04FF00009002E01D0002413E0C7F83B
:1044F0000090CAF800907846CBF800000020BDE894
:10450000F09F295D08EB0400FFF7FFFE000601D5D0
:104510003868F4E7641CB442F3D3C7F80090CAF8D3
:1045200000907846CBF800000020E8E72DE9F34F33
:10453000C3B005460024DFF86480DFF86490DFF83C
:1045400064A0002742A91448FFF753FE58B1822007
:10455000C8F800002120C9F800007846CAF8000019
:10456000822045B0E7E69DF80801800701D4FEF7F8
:1045700060FE02208DF8040028098DF8050004EB88
:1045800005108DF806008DF8077044980CE00000C7
:104590000080092000000940A08601007000001082
:1045A000740000107800001000EB04214FF48072BA
:1045B00002A8FBF77DFE00BF00BF00BF00BF00BF29
:1045C00000BF00BF00BF00BF00BF00BF00BF00BFF3
:1045D00000BF00BF00BF00BF00BF00BF00BF00BFE3
:1045E00000BF00BF00BF00BF00BF00BF00BF00BFD3
:1045F00000BF00BF00BF4026DFF8E0B3CBF81C606F
:104600004FF4827101A8FEF74AF8CBF8186000BF9A
:1046100000BF00BF00BF00BF00BF00BF00BF00BFA2
:1046200000BF00BF00BF00BF00BF00BF00BF00BF92
:1046300000BF00BF00BF00BF00BF00BF00BF00BF82
:1046400000BF00BF00BF00BF00BF00BF00BF641CB1
:10465000E4B2102CFFF476AF42A9E148FFF7C9FDA0
:1046600050B18220C8F800002120C9F80000784627
:10467000CAF80000822074E7FEF724FEC8F8007034
:10468000C9F800707846CAF80000002069E72DE9F3
:10469000FF5F894616460024DFF84883DFF848B3F9
:1046A000002E27D04FF4805501462A466846FBF776
:1046B000F5FDDDE90001CDE90201284600F08EFBA1
:1046C0000746380021D0A246351B0398C0F580501C
:1046D000A84200D20546B5F5805F21D03946029840
:1046E000FFF77FF8E0B1384600F050FBD8F8000043
:1046F00004B004E78620C8F800000920CBF80000C9
:104700007946BA4801608620F2E78220C8F80000A6
:104710002220CBF800007946B44801608220E7E708
:104720000298FEF7E4FF28B1384600F02FFBD8F8D6
:104730000000DDE7039809EB040138442A46FBF743
:10474000B7FD2C4439460298FFF7F0FE28B13846F1
:1047500000F01CFBD8F80000CAE70298401C029049
:10476000CDF80CA0B442AFD3384600F00FFBC8F828
:1047700000A0CBF800A079469C4801600020B7E774
:104780002DE9F04F89B00D46DDF8489092461F465E
:104790000024DFF85082B9F1000F4DD04FF480565D
:1047A0000146324601A8FBF779FDDDE90101CDE9BB
:1047B00005013246691C01A8FBF770FDDDE9010126
:1047C000CDE903013246514601A8FBF767FDDDE95B
:1047D0000101CDE90701A346A9EB04050898C0F53E
:1047E0008050A84200D20546089838B1059907982C
:1047F00088427DD1069908988842FAD14FF48050BA
:1048000000F0ECFA0646300021D00599079888425E
:1048100077D106990898884273D1DDE90702000331
:104820003146FEF7A4FE00061CD5304600F0AEFA75
:10483000D8F8000009B07EE58620C8F800006A4874
:10484000092101607946694801608620F2E78220EB
:10485000C8F800006448222101607946634801607D
:104860008220E7E703990798884211D1DDE9031018
:1048700000EB01300499C1F580523144FEF777FE18
:10488000000605D5304600F081FAD8F80000D1E7DF
:104890000798FEF72CFF000605D5304600F076FAA3
:1048A000D8F80000C6E70898391930442A46FBF7C3
:1048B000FFFC08983146421907980003FFF707FEEE
:1048C000000605D5304600F061FAD8F80000B1E7DF
:1048D00003990798884259D1DDE9031000EB0130B4
:1048E0000499C1F580523144FFF7F1FD000601E063
:1048F00050E006E04AD5304600F048FAD8F800000B
:1049000098E703990798884211D1DDE9031000EB7D
:1049100001300499C1F580523146FEF728FE0006A9
:1049200005D5304600F032FAD8F8000082E7079843
:10493000FEF7DDFE000605D5304600F027FAD8F870
:10494000000077E739190AEB04002A46FFF7BFFD9C
:10495000000605D5304600F019FAD8F8000069E7DE
:1049600003990798884211D1DDE9031000EB01306B
:104970000499C1F580523146FFF7A9FD000605D51F
:10498000304600F003FAD8F8000053E7304600F054
:10499000FDF90AE039190AEB04002A46FFF797FDF2
:1049A000000602D5D8F8000044E72C440798401CC4
:1049B0000790CDF820B04C45FFF40EAFC8F800B01A
:1049C0000948C0F800B0794608480160002031E786
:1049D0004FF4800070474FF48050704700800920EA
:1049E000A086010070000010740000107800001014
:1049F00000207047B14982200860B1492120086039
:104A00007846B049086082207047AC49822008602F
:104A1000AB49222008607846AA4908608220704786
:104A2000A64982200860A649222008607846A54948
:104A300008608220704738B50020009000BF00BF9A
:104A400000BF00BF00BF00BF00BF00BF00BF00BF6E
:104A500000BF00BF00BF00BF00BF00BF00BF00BF5E
:104A600000BF00BF00BF00BF00BF00BF00BF00BF4E
:104A700000BF00BF00BF00BF00BF00BF4024924D79
:104A8000EC619F20FDF704FE0020FDF701FE8DF88C
:104A900000000020FDF7FCFD8DF801000020FDF76F
:104AA000F7FD8DF80200AC6100BF00BF00BF00BF82
:104AB00000BF00BF00BF00BF00BF00BF00BF00BFFE
:104AC00000BF00BF00BF00BF00BF00BF00BF00BFEE
:104AD00000BF00BF00BF00BF00BF00BF00BF00BFDE
:104AE00000BF00BF00BF00BF784A0098811A904203
:104AF0001AD009DC11F5802016D0B0F5803F13D014
:104B0000B0F5003F0BD10FE0714808180AD0714989
:104B100040180BD07049C84201D1022400E00024A3
:104B2000204638BD0224FBE70324F9E70424FFF7FD
:104B300074FBF5E769480078002805D0684900EB68
:104B4000C00051F8200000475C49822008605C49A1
:104B50002120086078465B4908608220704770B564
:104B6000FFF769FF5D490870554D564E534C50B1E3
:104B70005B4900EBC00001EB8000806880470006C5
:104B800009D5206870BD82202060212028607846E9
:104B90003060822070BD0020206028607846306040
:104BA000002070BD2DE9F0414C4B454D454E1B7822
:104BB000424C002B0CD09AB1494F03EBC30307EBD7
:104BC00083031B699847000612D52068BDE8F08171
:104BD0008220206021202860784630608220F5E71E
:104BE0008620206009202860784630608620EDE726
:104BF000002020602860784630600020E6E72DE93C
:104C0000F041364B2E4D2F4E1B782C4C002B0BD0E9
:104C100092B1334F03EBC30307EB83039B699847C0
:104C2000000611D52068D1E782202060222028606C
:104C3000784630608220C9E78620206009202860FD
:104C4000784630608620C1E70020206028607846E2
:104C500030600020BAE7F8B5DDF818C01F4C184ED8
:104C6000184F2478154D002C10D0BCF1000F15D032
:104C7000CDF800C0DFF868C004EBC4040CEB84047A
:104C8000E469A047000611D52868F8BD8220286095
:104C900022203060784638608220F8BD8620286067
:104CA00009203060784638608620F8BD00202860F2
:104CB0003060784638600020F8BD000070000010B9
:104CC000740000107800001000800920C220180035
:104CD00003FBD6FF00FFFEFF0001F8FF28010010D4
:104CE0005C540000064C074D06E0E06840F001030C
:104CF00094E8070098471034AC42F6D3FBF7F6F976
:104D0000345500005455000030B50B4601460020D4
:104D10002022012409E021FA02F59D4205D303FA7D
:104D200002F5491B04FA02F52844151EA2F10102FE
:104D3000F1DC30BD30B58C1810F8012B12F00F03E8
:104D400001D110F8013B120906D110F8012B03E044
:104D500010F8015B01F8015B5B1EF9D101E001F87D
:104D6000013B521EFBD1A142E6D3002030BD02E040
:104D700008C8121F08C1002AFAD17047002001E0BC
:104D800001C1121F002AFBD17047000010B5002896
:104D900021D0114B0022001F196803E0814203D883
:104DA0000A4649680029F9D152B11368841A9C4215
:104DB00004D1006818441060104602E0506000E022
:104DC000186039B102680B1A934203D10B681A4478
:104DD00002604968416010BD2C010010F0B50B3035
:104DE000154D20F007010024144A0FE003688B42A0
:104DF0000BD38B4205D95E1A43184768C3E9006795
:104E000000E04368136002C004E0021D106800283F
:104E1000ECD12046002802D1286808B10020F0BD5E
:104E2000064A07481060074A121A22F00702C0E932
:104E3000002401202860D7E7300100102C01001069
:104E4000741D0010708D001000050F0A1B1E141138
:104E500033363C39282D272263666C69787D77725A
:104E600050555F5A4B4E4441C3C6CCC9D8DDD7D24A
:104E7000F0F5FFFAEBEEE4E1A0A5AFAABBBEB4B13A
:104E800093969C99888D878283868C89989D97922A
:104E9000B0B5BFBAABAEA4A1E0E5EFEAFBFEF4F11A
:104EA000D3D6DCD9C8CDC7C240454F4A5B5E54510A
:104EB00073767C79686D676223262C29383D3732FA
:104EC00010151F1A0B0E040103060C09181D1712EA
:104ED00030353F3A2B2E242160656F6A7B7E7471DA
:104EE00053565C59484D4742C0C5CFCADBDED4D1CA
:104EF000F3F6FCF9E8EDE7E2A3A6ACA9B8BDB7B2BA
:104F000090959F9A8B8E848180858F8A9B9E9491A9
:104F1000B3B6BCB9A8ADA7A2E3E6ECE9F8FDF7F299
:104F2000D0D5DFDACBCEC4C143464C49585D575289
:104F300070757F7A6B6E646120252F2A3B3E343179
:104F400013161C19080D07020000211042206330BF
:104F50008440A550C660E770088129914AA16BB1D1
:104F60008CC1ADD1CEE1EFF1311210027332522279
:104F7000B5529442F772D662399318837BB35AA321
:104F8000BDD39CC3FFF3DEE3622443342004011449
:104F9000E664C774A44485546AA54BB52885099571
:104FA000EEE5CFF5ACC58DD5533672261116300619
:104FB000D776F6669556B4465BB77AA719973887C1
:104FC000DFF7FEE79DD7BCC7C448E5588668A778D9
:104FD0004008611802282338CCC9EDD98EE9AFF911
:104FE000488969990AA92BB9F55AD44AB77A966AB9
:104FF000711A500A333A122AFDDBDCCBBFFB9EEB61
:10500000799B588B3BBB1AABA66C877CE44CC55C88
:10501000222C033C600C411CAEED8FFDECCDCDDDB0
:105020002AAD0BBD688D499D977EB66ED55EF44E58
:10503000133E322E511E700E9FFFBEEFDDDFFCCF00
:105040001BBF3AAF599F788F8891A981CAB1EBA154
:105050000CD12DC14EF16FE18010A100C230E320D0
:105060000450254046706760B9839893FBA3DAB378
:105070003DC31CD37FE35EF3B1029012F322D23220
:105080003542145277625672EAB5CBA5A895898548
:105090006EF54FE52CD50DC5E234C324A014810470
:1050A0006674476424540544DBA7FAB79987B89718
:1050B0005FE77EF71DC73CD7D326F2369106B016C0
:1050C00057667676154634564CD96DC90EF92FE9D8
:1050D000C899E9898AB9ABA9445865480678276810
:1050E000C018E1088238A3287DCB5CDB3FEB1EFBB8
:1050F000F98BD89BBBAB9ABB754A545A376A167A60
:10510000F10AD01AB32A923A2EFD0FED6CDD4DCD87
:10511000AABD8BADE89DC98D267C076C645C454CAF
:10512000A23C832CE01CC10C1FEF3EFF5DCF7CDF57
:105130009BAFBABFD98FF89F176E367E554E745EFF
:10514000932EB23ED10EF01E005EBCE2613FDD83C5
:10515000C29C7E20A3FD1F419DC3217FFCA2401E57
:105160005F01E3BD3E6082DC237D9FC1421CFEA047
:10517000E1BF5D0380DE3C62BEE0025CDF81633D37
:105180007C22C09E1D43A1FF4618FAA427799BC527
:1051900084DA3866E5BB5907DB856739BAE4065817
:1051A0001947A5FB7826C49A653BD987045AB8E607
:1051B000A7F91B45C6987A24F8A6441A99C7257BF7
:1051C0003A6486D85B05E7B98CD2306EEDB3510FE7
:1051D0004E10F2AC2F7193CD114FADF3702ECC92D7
:1051E000D38D6F31B2EC0E50AFF1134DCE90722CC7
:1051F0006D33D18F0C52B0EE326C8ED0530DEFB1B7
:10520000F0AE4C1291CF2D73CA947628ABF51749A6
:105210000856B4EA6937D58B5709EBB536688AD496
:1052200095CB2977F4AA4816E9B7550B88D6346A86
:105230002B7597C94A14F6A8742AC896154BA9F776
:10524000B6E80A54D7896B35EB3C904D53444F5325
:10525000352E3000020201000110000004F80C009D
:10526000010001000000000000000000000029EF24
:10527000BEADDE41544F4C20465072696E744641BB
:1052800054313220202000000000000000100000F7
:10529000002000000030000000400000005000002E
:1052A000006000000070000000800000009000001E
:1052B00000A0000000B0000000C0000000D000000E
:1052C00000E0000000F0000000000100008001008C
:1052D00000000200008002000000030000800300C4
:1052E00000000400008004000000050000800500AC
:1052F0000000060000800600000007000080070094
:10530000FF0F0000FF1F0000FF2F0000FF3F000005
:10531000FF4F0000FF5F0000FF6F0000FF7F0000F5
:10532000FF8F0000FF9F0000FFAF0000FFBF0000E5
:10533000FFCF0000FFDF0000FFEF0000FFFF0000D5
:10534000FF7F0100FFFF0100FF7F0200FFFF02005F
:10535000FF7F0300FFFF0300FF7F0400FFFF040047
:10536000FF7F0500FFFF0500FF7F0600FFFF06002F
:10537000FF7F0700FFFF070012011001000000403F
:1053800051C2031300010420480109022000010159
:1053900000803209040000020806506207058202FC
:1053A0004000000705020240000000040309041C3D
:1053B00003410054004F004C00200020002000203A
:1053C000002000200020002000200028034600507C
:1053D00000720069006E007400200046006C0061DD
:1053E0000073006800200020002000200020002022
:1053F0000020001A034600690072006D007700610A
:10540000007200650030003000300030000E034DA7
:105410000065006D006F0072007900007F200000C1
:105420000000000043260000000000000000000013
:10543000000000000000000000000000000000006C
:10544000000000000000000000000000000000005C
:10545000000000000000000000000000F149000012
:10546000F1490000F54900000B4A0000F549000031
:105470000B4A00000B4A00000B4A0000214A0000C2
:10548000F1490000F1490000F54900000B4A000015
:10549000F54900000B4A00000B4A00000B4A0000CF
:1054A000214A0000754000007B400000453E00009E
:1054B0007F3F0000CD3A0000033B00009136000022
:1054C000F53B0000814000009D300000A33000004B
:1054D000912A00007F3F0000CD3A0000172D000008
:1054E000CF440000352E0000A9300000D149000053
:1054F000D7490000453E00007F3F0000CD3A000044
:105500008F460000CF44000081470000814000002A
:10551000000000000000000000000000000000008B
:10552000000000000000000000000000000000007B
:10553000000000005455000000000010340100007D
:10554000344D00007C550000340100103C9C0000EC
:105550007C4D0000BD41544F4C20465072696E7422
:1055600028054AD4284B3D0276102C0E270780C30D
:10557000C90100879303044D6CDC0200E69E9A8EFD
:105580008BA428DDBAE6078666C4394EBABF10F18F
:10559000FF7214A58DB6A5AB1FF4C54C5500250CA4
:1055A000E61AAE5F15E804A29F141266A5A00E9E2F
:1055B0002B2F93A2B415149F8D6D4C1EF1CE69054F
:1055C000B6380581C36E469DB9146361B5A27B4CA4
:1055D000131B5932D2F6641FCA89ABEC4B0ADEDFCB
:1055E000688F94FDE96C2BAFE7EE24D2EEEBB31C91
:1055F0003F6978A60FB0A02A898F8824F725C7E4D1
:105600008F3CE6FCC61193DA1C6C07E88C19153D3B
:10561000CA03DE3322940AD64A497B17C1B337E165
:1056200014B76F42FF9EBE3755A8D7C2CD7A3074EB
:105630000BBBE9F553FB3A7BC048EF485AC490389E
:105640002D721A72196A2E47D2C2512B51B3D8E566
:10565000BC5F762EA9D65428690F41ED0246260577
:1056600037ED5BF328450BDB9E35BBEC52E468BDA0
:1056700062EA581B4EDFE6C713B00E5CEDFD99657C
:10568000FBB54B04B3329D65A2060BD1C4B2E23D1B
:10569000230948297A81535A0F218727FA5EA47A71
:1056A000753CA77F08240207159E24CBBB5D8A8129
:1056B000C4D1AA499C72AA3134FD3ED6DE36D74207
:1056C00032E8111C977F5748EC45CAF38F320D6DB5
:1056D000F8BD9CD9CCE43AFEAE707CBE200BB3552D
:1056E0002DCDC9537570F901009DE95885EF4378B8
:1056F000ED028499BD0A34B7149690CA2F865A7A5F
:10570000B004DF6D1376D31025DA0A3F99280D5BBC
:10571000788C29ED4C5E47CE98F91C1ACB54F4C412
:105720007135469837F8E06243FE938169164C6400
:105730000103ACA6F0708F13EA6F9AFBD608A01293
:1057400074F375B24B07BE18C4866298907CBB5B3D
:10575000CC4F02013D971E5862AB15A97227AAC310
:1057600008BC181F13EFBAF628AB30EF235DF26BBD
:105770009155A93D21B891DBB9AF5C1E668A45936E
:105780008B869D888250FC1DDB6D6E101986EA5B4E
:10579000DF72AC759AD732C7DF78E0BB7E6F856A5F
:1057A00081BD706875DAFC3A4A4BD4C40832D7C25E
:1057B0002E2E2E71646BB08689DCC94BE7DADD8949
:1057C000E0CD7F6CFA74FF4BE4A2B679A0147ADBCB
:1057D000F25D7373160B0035F77C02F711E53EDEC0
:1057E000A2E5E8B62BAF483A1929CC1E159DC28414
:1057F0002CE034B38E6C5E76A830AC6DF4307FCD87
:105800003E0BA6D828F1F9F167B54F5E0BA769C327
:10581000E6DFACECDF0689D9B5E0D5C22DDCD5DA00
:10582000B5D83D38D3C1CD2EF188D8EF7BFAB49BE3
:10583000D40E076664310702280BD616F7DD3E98B2
:105840001C0A31532B6768D0824D37C8097312A6E2
:10585000675B93B2209E84B75E49CAE8853A24A864
:10586000B2F3E949B8BAA358A0EA313DD63E6D1B60
:10587000BF09DF30124AD3FBD0655BC12B939789F8
:1058800042FB58AC29B241CEA94E924CCDBA5BBB7B
:1058900025E9F6A233597BFB99805183A0F001835F
:1058A000AC6470523BA43B87FADEE4F4B2BD02E67E
:1058B000F0F037C5850B9D94E1F7A112E01416BBFB
:1058C0003124A024D97AEA12CE98A74A1F652D3632
:1058D0001E094BB00C52355BADC9B316ECB6D339CB
:1058E000FE93F749F4A65F475EFF46BBC38257921B
:1058F000A6BFBABA4902274975E9F3A4A36E0EC13F
:10590000CFE5CDEBE0FFFFEB43B485D2B757AD8BCE
:10591000C53D3ADAAB45912354DAC8164EEEF5C6CA
:105920002CA06F2CB2DD42380B543AE407AF0B08C1
:105930004E0825F167540BBEAC189652FECBC8C674
:1059400069F2E193FCAFB39928A0C4CC9FCC820E3E
:1059500047B6282EA84E23201FFBC46E9AD50E06EC
:105960002992F6B303FB261E39CFAAF1DC7E14651B
:1059700032612113ECA039FC58A8D78D3757B227D4
:10598000E3872BC896721EBB65200D261DAE088AC4
:1059900024EC57BE8191BD3960FA0E9EB44872B3B3
:1059A00065D90E1643BE72926B0E9C3207C15D30F4
:1059B0008FBEB80808E34733F69E245B3FED535F84
:1059C0007B5593A0795475876678E91630C4912F7A
:1059D00051AF7B1FAE6DDB6187528C511C7910C1BA
:1059E00050A92DAC5C2EEEBF9D44533A9B2006B7C8
:1059F0000FC3F95E38006AAB19EE69F9FFA8F2D956
:105A00000A732478CBE00459CF7456EDD2B307DF84
:105A1000637B30EA5F0A1A2A090E409587CA2791EC
:105A200013205F2C3FE1F0101ECDD6F25B6CE980B5
:105A300073DC7A81432789181CBDA00A25C3EF2C8B
:105A40003C96223A38BBAC7D6B55CF4C8F65DA095A
:105A5000C648CBF2D68BE6DB4EA59D9A73131AFC93
:105A6000E956ECB8D7B28BFADBD33B2D0A26E41209
:105A7000872B03D92EBF232DE789E8665134962F53
:105A80000CE478E9DDA4783BA40BD94695FF698E38
:105A9000B28E5D2EB764C692B59C4EC55A149B78E3
:105AA000DA1CDFE5AEFFD74311EEEC4DA7B1CE9F78
:105AB000392A7FEEDB1A3108FB4153202781941DE0
:105AC000881FD18494C09BF990A7C5DC28E972D9BE
:105AD000272B6565879F465B8415BC447892D32B42
:105AE0005A12B2F5D47E65A36C5E4DA3979F3A48D7
:105AF0005288B9E0F60B7EAF52F552E4FF9732813F
:105B0000BBC81F9F66537FFF95BFAFA37442EA0BCC
:105B10002C87D89CA6A3C97EEA51938E1C10CE7800
:105B20004E325055057BA4EF88D8D7F6DD17B5BAAD
:105B3000A4C29BCC774C50E7BCA119004FC4AB6DFD
:105B40000B7BE1B2A421B8413EA0A3DA8E2D83786D
:105B5000EF4C843BE80C717C8ABB32E96B1526372D
:105B6000DECE3EB98660CE823CB245262C0A3B375B
:105B7000FC5F22C4B84D7FC2775BF7FD39FB204440
:105B80006ED7092C88420CDCBB9DB1780DBC6CDB58
:105B90005B514BEE7C2138AB72E1D886DE80809B76
:105BA0004AF559AC386D637B0E9391881F488B83FF
:105BB0001D2398BC4630B49792BB61E17A3950A559
:105BC000360B305FA6D314D86F964280F8170A8838
:105BD000C1994525A47AAF2A3DA8863DF6EDA425B6
:105BE0006CD706D6B97B6FE976A47244936B27BC59
:105BF0006D5FC478AC373C55BD198F854CB20A0D2A
:105C0000AA4325A16255D27CA30D4BD9B376B6F534
:105C100035AF3C9F7AABF9B7A6D661270672998952
:105C20008C4DF459C0A9393279E6CC4B7D7874F4A7
:105C3000D0610C483C93FB9443C982FB3B93C06604
:105C40003B728300972934BD143D71D6946D17447F
:105C50007F65F57934C337547BAF808681A81CFEFD
:105C6000E476EB4F1622BB5D47DD400FB0DA46CE3F
:105C700034D8C3C63B1FED982C9C53A8FCE624588F
:105C800031A77ED9BB7777FAD4D1869528B8AF787B
:105C90007B5C47AAB0567C2ED3C9EBF5D122232FCB
:105CA000B8A3496754FB437E5C17F8C39E51803903
:105CB000064E32B0F2AE9748F7F496723C614D53FF
:105CC000C108B248A5DDDBF07DF2057A4B53A08216
:105CD000DD46A74F81FE1D3AECF6E91B47AC51307B
:105CE0003E21A8B989F5EF824CA128D01EB146000B
:105CF000102A966F3B1FA48BC31458403652681B62
:105D00004836D8EFFDA9F776D6B319A1505E839F28
:105D100090A7F097DCB008855F59CAE4BBDEEA3093
:105D20007D61EE9FB75687197B9884127B312102E3
:105D3000F43656E0E3E6E2842000B1AA2C29877A03
:105D40005E7182BBE192B1E893FDAFDABC58399441
:105D5000E6713BC7E4C8B1F8085E81EC81161FA369
:105D6000EA912B6DB4706C53C917ACFBDF99AE5A36
:105D7000D0308031A3C92451B6AF0B44EC03F105F8
:105D8000B148106D090B1F7E7918B9A561CED216E6
:105D90005759D9FB031DBAFC293BFB1994035A49F7
:105DA000E3ACF1D5015B991CF2863ED46A31359C97
:105DB000E653DC00A60CA2C80FBD3BD3802A918B12
:105DC000DF1E70F705B41F90A15EE6075E0700F9BD
:105DD0008ACA7DABA4691FB0A706AB709F012630AD
:105DE000B38D81225A30267589C2A3DF06B6050B12
:105DF00077FF8B63A28B525CBEEFC7F6D3BB4BFA27
:105E0000EAAF83C885BB114C870D06771A031B2F99
:105E1000FE5F8D09E2F4D68D25E44DAE8F24D79335
:105E200042973B1D4647456F89AD6A1CC0EC64AC88
:105E300053C35BF7FF19924783E71300DB4414FF5A
:105E40001FA6128F589E8C15B7C4659B07621D70E4
:105E50006A278F7B77F7320DA78F2404CD48B03C9B
:105E600056E535E5A4A7F91333230C145B6EDD3139
:105E70005985232B5D830D87640EE104392EDF08DD
:105E800039AC8464EFA74C6BB21F499412D88ADBFB
:105E9000180FB386E66B4E7C6DA593A717EE128E96
:105EA000FF063571F1D1CF97E128DE45B1D1888663
:105EB000CC30089BC83D5495E6EC4E9D3FFE281B18
:105EC00009451A6FE4C244249A20B3AB77C64E0743
:105ED000B9EA37AA56703F4013DD35A2D2DD95D618
:105EE000587A9937056FF7A6FAD16B8D82CD2F1AA4
:105EF000C99CA55E73EC9BB09AB3B9F99C1FF627B9
:105F0000BE847890CEFACFFA3FE4044B84E4318D1E
:105F1000376053194092B6EE5BF84E4B040BBCD081
:105F20001685F31E9B948BB57D786C43227B269A55
:105F300068B865540DA270913CE866088101BBB257
:105F40006275D8366C1966EA2B6214A95455D7CFFE
:105F5000CDCFDC0A04852491FA6EF99627D18D867F
:105F60007C93D4369DBBB566F9B548CEC1C43E8A94
:105F70005191AE3E1A07CEE7FDA319A459854CA74F
:105F80006C7DC4C5F87732497200E80AD27D641E80
:105F9000E606F387AEE5E03342EA6A17AFFDA5D91E
:105FA000AA4DCA642C5D84C68A4DA0C66BD36A34E0
:105FB0006ECEF313E66A7A77E3BAD6342F1021C592
:105FC0006AC53716D176024AB90B96BB67653C01A4
:105FD000507E409C7670883C474E0D4D75487E60E3
:105FE000D79A8369CFF4B91EF7B0FB2AA2C75184B0
:105FF000EA25B789AF37399406F75769E9E6D26ED3
:00000001FF
